:1000000018308A00012B0000FF00030E8301A100BD
:100010000A08A0008A010408A2007708A300780853
:10002000A4007908A5007A08A6007B08A70083131E
:1000300083128B1D1D280B1840288C308400801ED5
:1000400023288C1A43288C308400801C29288C1883
:1000500046288B1E2D280B194928220884002308C6
:10006000F7002408F8002508F9002608FA002708F8
:10007000FB0020088A00210E8300FF0E7F0E09007E
:100080008A110A1213298A110A1600288A110A12E3
:100090009E2B8A110A1237290A108A100A11820728
:1000A000483465346D3469344F3453342034563415
:1000B000253464342E342534643420342C342034F4
:1000C0004B342D345434653461346D34203453341E
:1000D0002E3441342E3420342834203441346C34CE
:1000E0006534783461346E34643472346534203469
:1000F00043346F346C346F347434203429342034F6
:10010000203400340A108A100A1182073034313446
:100110002D346D34613469342D3430343734003447
:100120000A108A100A118207313431343A343334D8
:1001300039343A343434363400340A108A100A110F
:10014000820745342D344D34613469346C342034A5
:100150003A34203469346E3466346F344034683451
:1001600065346D346934733473346F346E342E34C3
:1001700063346F346D340D340A340D340A34003472
:100180000A108A100A11820755346E346B346E34AB
:100190006F3477346E34203443346F346D346D34BF
:1001A00061346E34643420343F3421340D340A34E5
:1001B00000340A108A100A11820762342C34483441
:1001C00065346D3469344F3453345F3476345F347E
:1001D000253464342E34253464340D340A34003428
:1001E0000A108A100A11F73E03188A0A8200443462
:1001F000E9346D3461347234723461346734653497
:10020000203465346E3420346D346F346434653496
:10021000203449346E347434653472346E34653449
:100220000D340A340034AD1C3329F930F700F70BD4
:100230001729000000000030061A0130003A031DA3
:100240003329B2012D13061E2D17B20A8B1110305F
:10025000F80006389200BB30831692008312910199
:1002600083168C1483120B108A110A122D28B80AD7
:100270003808053C031D4529B8010130B4070318AF
:10028000B50A0319B60A0319B70AAA1B57292A087F
:100290000F3C2C07F700F71B542977080E3C031876
:1002A00054290810881056290814881067292A082C
:1002B000003C0F3C2C07F700F71B652977080E3C24
:1002C0000318652908108810672908108814AB1BCB
:1002D00079292B080F3C2C07F700F71B76297708A4
:1002E0000E3C031876290811881178290815881101
:1002F00089292B08003C0F3C2C07F700F71B8729A6
:1003000077080E3C031887290811881189290811DC
:100310008815AC0A2C080F3C03188F29AC0139084A
:10032000013A0319BB29023A0319E929093A0319C9
:100330000D2A063A0319502A033A03198A2A1B3A4E
:1003400003198F2A023A0319D22A0F3A03190D2BE7
:100350003A3A03193E2B473A0319432B1C3A031927
:10036000442BF43A0319452B2C3A0319462B683ACF
:100370000319472B4E2B2D1CE8293030F8001F089D
:10038000C73978049F001330F700F70BC529000028
:1003900000001F151F19CA291E0883160317D8004D
:1003A0003830F800831203131F08C73978049F0000
:1003B0001330F700F70BDA29000000001F151F1992
:1003C000DF291E0883160317D9008312031386142E
:1003D0004E2B2D1C0C2A1F151F19EC291E088316E5
:1003E00003175902E1003030F800831203131F088D
:1003F000C73978049F001330F700F70BFD29000080
:1004000000001F151F19022A1E0883160317590220
:10041000E0008312031386104E2B2D1C4F2A083048
:10042000F8001F08C73978049F001330F700F70B56
:10043000172A000000001F151F191C2A1E0883160A
:100440000317D3000030F800831203131F08C739C5
:1004500078049F001330F700F70B2C2A00000000EF
:100460001F151F19312A1E0883160317D2001030DA
:10047000F800831203131F08C73978049F00133054
:10048000F700F70B412A000000001F151F19462A2C
:100490001E0883160317D4008312031306154E2B70
:1004A0002D1C892A1F151F19532A1E08831603178E
:1004B0005402DC000830F800831203131F08C73908
:1004C00078049F001330F700F70B642A0000000047
:1004D0001F151F19692A1E08831603175302DB0014
:1004E0000030F800831203131F08C73978049F00F7
:1004F0001330F700F70B7A2A000000001F151F19B0
:100500007F2A1E08831603175202DA008312031390
:1005100006114E2BBA08031D8E2A88174E2B2D1C50
:10052000D12A2030F8001F08C73978049F00133003
:10053000F700F70B992A000000001F151F199E2ACB
:100540001E0883160317D6002830F8008312031301
:100550001F08C73978049F001330F700F70BAE2A45
:10056000000000001F151F19B32A1E088316031769
:10057000D7001830F800831203131F08C739780416
:100580009F001330F700F70BC32A000000001F156F
:100590001F19C82A1E0883160317D50083120313D8
:1005A00086154E2B2D1C0C2B1F151F19D52A1E0826
:1005B000831603175502DD002030F8008312031361
:1005C0001F08C73978049F001330F700F70BE62A9D
:1005D000000000001F151F19EB2A1E0883160317C1
:1005E0005602DE002830F800831203131F08C739B3
:1005F00078049F001330F700F70BFC2A000000007E
:100600001F151F19012B1E08831603175702DF0041
:100610008312031386112D164E2B83160317E20146
:10062000831203130718192B83160317E20A831288
:10063000031383160317E301831203138718252B73
:1006400083160317E30A8312031383160317E401C7
:10065000831203130719312B83160317E40A83123D
:10066000031383160317E50183120313871A3D2B27
:1006700083160317E50A831203134E2BBA08031DD2
:10068000422B88134E2B4E2B4E2B4E2B4E2BB9014B
:10069000BA0A3A080A3C031CBA014E2BB90A0B11DC
:1006A0008A110A122D2801303102EF3E0318862BE1
:1006B000113E892B0530AA000A30AB00862B0A3088
:1006C000AA00AB00862B0A30AA000530AB00862BAF
:1006D000F630AA000A30AB00862BAA01AB01862BAC
:1006E0000A30AA00F630AB00862BFB30AA00F630A9
:1006F000AB00862BF630AA00AB00862BF630AA00A2
:10070000FB30AB00862B862B862B862B8A110A1298
:10071000552C0A148A140A1182075A2B5F2B632B5B
:10072000682B6D2B702B752B7A2B7E2B862B862BB3
:10073000832B862B862B862B842B852B0130320234
:10074000F33E0318602C0D3E652CAD13061EAD174D
:10075000AD1BB32B1030F8009200BB308316920013
:100760008C1083128B15602C2F10061E2F14602CFA
:10077000AF10061EAF14AF1CC62B1030F80092004D
:10078000BB30831692008C1083128B15602C2F11B6
:10079000061E2F152F1DD52B1030F8009200BB30F0
:1007A000831692008C1083128B15602CAF11061EDD
:1007B000AF15AF1DE42B1030F8009200BB3083164C
:1007C00092008C1083128B15602C2F12061E2F1690
:1007D0002F1EF32B1030F8009200BB3083169200CE
:1007E0008C1083128B15602CAF12061EAF16AF1E35
:1007F000022C1030F8009200BB30831692008C104F
:1008000083128B15602C2F13061E2F17602CAF132D
:10081000061EAF17602C3010061E3014602CB0106E
:10082000061EB014602C3011061E3015602CB0115D
:10083000061EB01500302F1B0130F700770EEA00BE
:10084000EA0DE030EA050030AF1B0130F700F70E8B
:10085000F030F70577086A04EC00003030180130FA
:10086000F700F70DF70DF70DF830F70577086C0472
:10087000EE000030B0180130F700F70DF70DFC3036
:10088000F70577086E04F000003030190130F700EA
:100890000310F70D77087004F2000030B019013032
:1008A0007204B100AD1D552C532BAD161030F8005D
:1008B0009200BB30831692008C1083128B15602C33
:1008C000B20A8C108A110A122D280A108A100A15F1
:1008D0008207A52BB42BB82BC72BD62BE52BF42BDB
:1008E000032C072C0B2C0F2C132C172C83162B08E6
:1008F000F8012A0203187F2C2A08F7008B2CF70135
:100900000830AC00AA0DF70D2B0877020318F7008A
:10091000F80DAC0B822C8312003420308316251E78
:100920003030A6002408F700A41F9D2CF709F70A11
:100930007708A4002D30A600A5172408AA0064306B
:10094000AB008312762477088316A4003030780732
:10095000A7002408AA000A30AB00831276243030A6
:1009600077078316A90030307807A8002608F7001B
:10097000A51DBC2CA51F2511251AC92CA51FE42CCB
:100980002519E42C7708A700A518E42C7708A800FF
:10099000E42C30302702031DE42C7708A700203018
:1009A000A600A51DD72C2511A514A51FA510303014
:1009B0002802031DE42C7708A8002030A700A51DFD
:1009C000D72CA510A51F2510251DEE2C2608831257
:1009D0000C1AEC2C8316E72C99008316A51CF82C16
:1009E000270883120C1AF62C8316F12C9900831613
:1009F000251C022D280883120C1A002D8316FB2CAF
:100A000099008316290883120C1A082D8316032DCA
:100A1000990000348316A00120088312D920831680
:100A2000A00AF70083120C1A172D8316122D9900B5
:100A30000B3083162002031D0C2D0130A4001F3043
:100A4000A50083128D242E300C1E242D99003330E6
:100A50008316A4001F30A50083128D240D300C1EB8
:100A60002F2D99000A300C1E332D99008A110A1679
:100A70003C2F65300C1E3A2D99002C300C1E3E2D5B
:100A800099002A088316A4000130A50083128D2442
:100A90002C300C1E492D99002B088316A400013020
:100AA000A50083128D240D300C1E542D99000A30A0
:100AB0000C1E582D99008A110A163C2F94138C1184
:100AC00083162308831293000230941B6E2D8C1D15
:100AD000672D00308316111B01308312F80000349B
:100AE000831691159119722D77189112771C911612
:100AF0001116111A792D83121308F8000034831689
:100B0000A41B972D0F30F700230EF7050A3077024C
:100B100003188D2D3030F7078F2D2408F70777083D
:100B200083120C1A952D8316902D990083160F3081
:100B3000A3050A30230203189F2D3030A12DA413E2
:100B40002408A307230883120C1AA82D8316A32DAB
:100B500099008A110A12E82D6A300C1EAD2D9900F9
:100B600003308316A0002008FD3C031CF22D111455
:100B70001118B82D01302002A200A30083125E25B7
:100B8000F808031DE92D8316A30183125E25831641
:100B900091149118C92D2008A30083125E25F70136
:100BA000702578088316A10011151119D52D013073
:100BB0002002A2002C3083120C1AE02D8316DB2DAC
:100BC000990083162208A3005730A40083127F2DBA
:100BD000EE2D831611151119EB2D83120230831699
:100BE000A007B32D0D3083120C1AF82D8316F32DA8
:100BF00099000A300C1EFA2D99008A110A163C2F12
:100C0000780883162008AA006430AB00831276248B
:100C100077088316A00078083030031D162EA11C1B
:100C2000222EA119222E211A2030192EA1112112B3
:100C30002114F807780883120C1A202E83161B2E15
:100C4000990083162008AA000A30AB00831276248C
:100C500077088316A00078083030031D352EA119BF
:100C60003E2E211C3E2E211A2030F80778088312D0
:100C70000C1A3C2E8316372E990083163030A007AD
:100C8000200883120C1A462E8316412E9900003438
:100C900071300C1E492E9900003041028316A000CD
:100CA000831242088316A1001830031C1930A102D8
:100CB0002108A20083120C1A5F2E83165A2E990067
:100CC000003041028316A000831242088316A1005F
:100CD0001830031C1930A1022008A20083120C1A3C
:100CE000732E83166E2E9900BC013C08073C031C32
:100CF000882EDA303C078400831700088316A00092
:100D000083120C1A852E8316802E9900BC0A752E2C
:100D1000BC013C08073C031C9C2ED2303C078400DD
:100D2000831700088316A00083120C1A992E8316CD
:100D3000942E9900BC0A892E3E080C1E9D2E990007
:100D40000030061801308316A00083120C1AAA2E58
:100D50008316A52E99008A110A163C2F83162508A2
:100D6000403C0318B82E413025020A3EA600BB2E97
:100D700030302502A6002608F800831200348C1EAD
:100D8000BF2E1A0883160317A000831203138C1AB0
:100D9000CC2E83160317C52E1A0883160317A1003D
:100DA0002008FA00210883120313C10018307A07C3
:100DB000C2008316031720080313A100031721089C
:100DC0000313A0001A30FA00FF30831203178D00BE
:100DD0007A088F00831603132008831203178C00F0
:100DE000831603132108831203178E0083168C17B2
:100DF0000C15831203130B08F8008B1383160317CB
:100E000055308D00AA308D008C14000000008C1825
:100E1000072F0C117808831203138B04BE01B01244
:100E200073300C1E112F99008A110A163C2F743052
:100E30000C1E182F99002C300C1E1C2F9900310805
:100E40008316A0000330A100831200260D300C1E73
:100E5000272F99000A300C1E2B2F99008A110A1691
:100E60003C2F8C1E312F1A0883160317A000831203
:100E700003138C1A3E2F83160317372F1A08831675
:100E80000317A1002008FA00210883120313C100F0
:100E900018307A07C20042081A3C0318532F1A3040
:100EA000C200FF30C10030121830C000BF0140083E
:100EB0004202031CA62F031D612F41083F020318A5
:100EC000A62F301A652F8812662F88168C1E662F63
:100ED0001A08BC008316A10183123C088316A000E7
:100EE00083124008FA003F0803178D007A088F002C
:100EF000831603132008831203178C008316031331
:100F00002108831203178E0083168C170C15831289
:100F100003130B08F8008B138316031755308D004D
:100F2000AA308D008C14000000008C18952F0C1135
:100F30007808831203138B041030B0063C080C1E93
:100F40009F2F9900BF0A0319C00A572F8812FF303C
:100F5000C200C10075300C1EAB2F99008A110A1611
:100F60003C2FFF30C200C10008130516AA01AB01D7
:100F7000081278300C1EBA2F99008A110A163C2FDD
:100F80007A300C1EC12F99000D300C1EC52F990010
:100F90000A300C1EC92F99008A0100288A110A16EE
:100FA0003C2F8316A00120088312C0208316A00ABC
:100FB000F70083120C1ADE2F8316D92F99001430F4
:100FC00083162002031DD32F83120034593084006E
:100FD000831300080319F92F0630F800F701F70B07
:100FE000EF2FF80BEE2F7B30F700F70BF52F800B70
:0C0FF000EC2F00342D1057182D14003485
:1010000031300C1E012899002C300C1E0528990047
:10101000831603172208303A831203130319172883
:10102000013A03193228033A03194D286828831618
:1010300006080138A000860000308312061801302F
:101040008316A000A4001F30A5008A1183128D24EE
:101050008A150D300C1E2A2899000A300C1E2E28E5
:1010600099006C28831606084038A00086000030DE
:101070008312061B01308316A000A4001F30A500B8
:101080008A1183128D248A150D300C1E4528990073
:101090000A300C1E492899006C28831606088038EF
:1010A000A000860000308312861B01308316A0004A
:1010B000A4001F30A5008A1183128D248A150D30DB
:1010C0000C1E602899000A300C1E642899006C28B8
:1010D0008A11D1278A156C288A110A163C2F3230C2
:1010E0000C1E702899000D300C1E742899000A30CF
:1010F0000C1E78289900831603172208303A8312B1
:10110000031303198A28013A03199F28033A031984
:10111000B428C92883160608FE39A000860030309E
:1011200003172402003A031D9B28831203130610A1
:101130009E2883160317831203130614CD288316E3
:101140000608BF39A0008600303003172402003A99
:10115000031DB028831203130613B3288316031745
:10116000831203130617CD28831606087F39A000C3
:101170008600303003172402003A031DC52883126D
:1011800003138613C82883160317831203138617C5
:10119000CD288A11D1278A15CD288A110A163C2F0D
:1011A000AA01AB0183160317D201D301D401D501E3
:1011B000D601D701D801D901DA01DB01DC01DD015B
:1011C000DE01DF01E001E101E201E301E401E5010B
:1011D00003130912F701F71DF82807308312810164
:1011E0008130840083130008C0390F3880008316D3
:1011F0006400813084000008C039770480008312C5
:1012000090010030F80092000030831692008312A3
:10121000970197019D019D012F3083168500303085
:101220008600A7308700003088000F30890010301A
:1012300083128500860187018801831681171F109C
:101240009F101F119F1183121F179F1783169F1343
:1012500083121F14F8009200BB3083169200831291
:10126000910183160108C039013881008312810180
:10127000B53090008F018E010530D9008A11E62724
:101280008A15C70147088A114C208A15C70AF7003A
:1012900077080C1E4929990008304702031D42298E
:1012A000A8018B1BA8178B1301308316A4001F30D5
:1012B000A5008A1183128D248A15A81B8B172E3046
:1012C0000C1E60299900A8018B1BA8178B133330C3
:1012D0008316A4001F30A5008A1183128D248A155D
:1012E000A81B8B170D30C80048088A114C208A159E
:1012F000C80AF70077080C1E7B2999003130480294
:10130000031D7429C70147088A1182208A15C70A5C
:10131000F70077080C1E8A29990009304702031D3F
:10132000832920300C1E9229990040300C1E9629EA
:10133000990020300C1E9A299900C70147088A118C
:1013400090208A15C70AF70077080C1EA529990076
:1013500008304702031D9E290D300C1EAD2999004F
:101360000A300C1EB1299900C70147088A119D2037
:101370008A15C70AF70077080C1EBC2999001E3091
:101380004702031DB5298B168B152D1DCA298316FF
:101390008C168312C0308B048A150A164B2BAD10A5
:1013A0005718AD1400342D1157182D150034AD11F8
:1013B0005718AD1500340330DA02031CEA295A30FD
:1013C0008400831300080319EA29E82900000000BB
:1013D000800BE62900345708D8005808003A031952
:1013E000F829013A0319772A033A0319F62A4A2BF6
:1013F0000830F8001F08C73978049F001330F70041
:10140000F70B002A000000001F151F19052A1E08EF
:1014100083160317D3000030F800831203131F084C
:10142000C73978049F001330F700F70B152A000026
:1014300000001F151F191A2A1E0883160317D20051
:101440001030F800831203131F08C73978049F0077
:101450001330F700F70B2A2A000000001F151F1990
:101460002F2A1E0883160317D400831203130615B0
:101470000230D9009530DA00DB21D90B3A2A1F154A
:101480001F19402A1E08831603175402DC00083077
:10149000F800831203131F08C73978049F00133024
:1014A000F700F70B512A000000001F151F19562ADC
:1014B0001E08831603175302DB000030F800831266
:1014C00003131F08C73978049F001330F700F70B88
:1014D000672A000000001F151F196C2A1E088316BA
:1014E00003175202DA008312031306114A2B20302D
:1014F000F8001F08C73978049F001330F700F70B76
:101500007F2A000000001F151F19842A1E08831659
:101510000317D6002830F800831203131F08C739B9
:1015200078049F001330F700F70B942A00000000A6
:101530001F151F19992A1E0883160317D700183084
:10154000F800831203131F08C73978049F00133073
:10155000F700F70BA92A000000001F151F19AE2A7B
:101560001E0883160317D500831203138615023055
:10157000D9009530DA00DB21D90BB92A1F151F19C4
:10158000BF2A1E08831603175502DD002030F8001D
:10159000831203131F08C73978049F001330F70024
:1015A000F70BD02A000000001F151F19D52A1E08AE
:1015B000831603175602DE002830F8008312031347
:1015C0001F08C73978049F001330F700F70BE62A8D
:1015D000000000001F151F19EB2A1E0883160317B1
:1015E0005702DF008312031386114A2B3030F800B4
:1015F0001F08C73978049F001330F700F70BFE2A45
:10160000000000001F151F19032B1E088316031767
:10161000D8003830F800831203131F08C739780444
:101620009F001330F700F70B132B000000001F156D
:101630001F19182B1E0883160317D90083120313D2
:1016400086140230D9009530DA00DB21D90B232B28
:101650001F151F19292B1E08831603175902E100B5
:101660003030F800831203131F08C73978049F0035
:101670001330F700F70B3A2B000000001F151F195D
:101680003F2B1E08831603175902E0008312031331
:1016900086104A2B0530D9008A11E6278A150034B6
:1016A000DA305707840083170008F8000034D708A1
:1016B000031D5C2B08125D2B08160034F701F8019E
:1016C0005E0803105F18F707F70CF80CDF18F70730
:1016D000F70CF80C5F19F707F70CF80CDF19F70790
:1016E000F70CF80C5F1AF707F70CF80CDF1AF7077E
:1016F000F70CF80C5F1BF707F70CF80CDF1BF7076C
:10170000F70CF80C0034D708031D882B0813892B1D
:1017100008170034D70803198F2B0512902B0516D4
:1017200000345708AA005808AB000034C701C801AC
:1017300048088A11F0208A15C80AF70077080C1E9D
:101740009F2B99001B304802031D982B003007186F
:101750000130F700770DC800C80DC80DF830C80576
:10176000003087180130F700F70DF70DFC30F70552
:1017700077084807C900003007190130F700031047
:10178000F70D77084907CA000030871A01304A0769
:10179000C7004708013A0319D42B033A03196A2DED
:1017A000063A0319B42DDC2DD7018A11FA278A15C0
:1017B000D701CF21D701D321D701D721D701EB21E1
:1017C0000130D700EB210230D70050237808C80041
:1017D0000430D70050237808C9000530D7005023C3
:1017E0007808CA000130D70050237808CB00D70111
:1017F00050237808CC0048081E3C031C012C003004
:10180000022C0130D7004C081E3C031C092C003070
:101810000A2C01305705D8004B081E3C031C122C23
:101820000030132C01305805003A03191A2C0130EE
:10183000D700572351084802003A031D212C0030DD
:10184000222C0130D80051084802D9005908053C23
:10185000031C2C2C00302D2C01305805DA004808D0
:10186000193C031C352C0030362C01305A05003A47
:1018700003193C2C56143D2C56104D084902003AD1
:10188000031D442C0030452C0130D8004D0849027E
:10189000D9005908053C031C4F2C0030502C013056
:1018A0005805DA0049081E3C031C582C0030592CFE
:1018B00001305A05003A03195F2CD614602CD6105B
:1018C0004E084A02003A031D672C0030682C013094
:1018D000D8004E084A02D9005908053C031C722C56
:1018E0000030732C01305805DA004A081E3C031CF6
:1018F0007B2C00307C2C01305A05003A0319822CD5
:101900005615832C561150084C02003A031D8A2CA0
:1019100000308B2C0130D80050084C02D9005908F7
:10192000053C031C952C0030962C01305805DA003C
:101930004C081E3C031C9E2C00309F2C01305A0585
:10194000003A0319A52CD615A62CD6114F084B0228
:10195000003A031DAD2C0030AE2C0130D8004F08EA
:101960004B02D9005908053C031CB82C0030B92C97
:1019700001305805DA004B081E3C031CC12C003016
:10198000C22C01305A05003A0319C82C5616C92C2E
:101990005612003056180130D7000530DE005708C7
:1019A000DF005E237808053CD8000030D6190130EE
:1019B000D9000A30DE005908DF005E23780858029B
:1019C000DA000030D6180130F7000310F70D770861
:1019D0005A07DB00003056190130F700F70DF70DFC
:1019E000FC30F70577085B02DC000030561A013046
:1019F000DD000630DE005D08DF005E2378085C074E
:101A0000D200003056180130D7000530DE005708EC
:101A1000DF005E237808053CD8000030D61901307D
:101A2000D9000630DE005908DF005E237808580729
:101A3000DA000030D6180130F700F70DF70DFC3052
:101A4000F70577085A02DB00003056190130F7001D
:101A50000310F70D77085B07DC000030561A0130E1
:101A6000DD000A30DE005D08DF005E2378085C02DE
:101A7000D3005308520203194C2D5308803AF70043
:101A80005208803A77020318492D0130D70083238A
:101A90004C2D0130D7008A235208D7005308D800B4
:101AA00091232830D7005708D9008A11E6278A15D4
:101AB000D7018323D7018A23D70157234B08CF00AF
:101AC0004C08D0004908CD004A08CE004808D10093
:101AD000DE2BDC2DC801C901D7018A11FA278A152E
:101AE000D701CF21D701D321D701D7210230D70089
:101AF000EB210630D70050230310780CCB000730C1
:101B0000D70050230310780C4B07C9000230D700D0
:101B1000EB210630D70050230310780CCB000730A0
:101B2000D70050230310780C4B07C8000230490738
:101B300048020319A82D031CA82D0330D700073035
:101B4000D8009123D70183230130D7008A23B22DF7
:101B50000730D7000330D80091230130D70083230A
:101B6000D7018A23862DDC2DD7018A11FA278A1501
:101B7000D701CF21D701D321D701D7210A30D700F0
:101B80000530D80091230430C800E130D9008A1113
:101B9000E6278A15C80BC52DFB30D700F630D800D4
:101BA00091230430C800E130D9008A11E6278A1554
:101BB000C80BD32DBE2DDC2D8A150A167E2BC70827
:101BC000031DE42D8812E52D88168A150A16B92BF7
:0E1BD000D2304707840083170008F800003465
:10200000F301F4018C1E1228A0302E0784008317E0
:102010008C1E08281A0880002E084E3C031C11282C
:10202000AE0A022801302E02A03E84008317000869
:102030000D3C031D3D2F831603172008423A8312DF
:10204000031303196C28063A03196F28013A031980
:10205000B8280D3A0319BB28013A0319D828033AC6
:1020600003192129063A03192429013A0319712970
:10207000033A0319202A013A0319A52A1F3A031922
:102080002A2B013A0319D92B033A0319DC2B013A05
:1020900003198B2C073A03198E2C013A0319912C42
:1020A000023A0319942C0F3A0319112D013A03191E
:1020B000142D033A0319C62D7C3A0319C92D0C3A85
:1020C0000319C12E0B3A03190E2F103A03192E2FA4
:1020D000033A0319332F382F0A120A2D0A168316D2
:1020E000031722082D3C031D922830302302003CA8
:1020F00083120313AA008316031725082D3C031D22
:102100008A2830302602003C83120313AB008F284C
:10211000831603173030250283120313AB00AB285C
:10212000831603173030220283120313AA0083168A
:10213000031724082D3C031DA62830302502003C3F
:1021400083120313AB00AB2883160317303024022D
:1021500083120313AB0064300C1EAC2899000D30C1
:102160000C1EB02899000A300C1EB42899003C2F90
:102170000A12392D0A163030831603172202003A4C
:10218000031DC828831203130812CB2883160317D4
:1021900083120313081668300C1ECC2899000D30EA
:1021A0000C1ED02899000A300C1ED42899003C2F10
:1021B00069300C1ED92899002C300C1EDD2899009E
:1021C0008316031762080313A4001F30A5000A1228
:1021D00083128D240A162C300C1EEC2899008316CD
:1021E000031763080313A4001F30A5000A1283120B
:1021F0008D240A162C300C1EFB2899008316031719
:1022000064080313A4001F30A5000A1283128D2452
:102210000A162C300C1E0A2999008316031765082C
:102220000313A4001F30A5000A1283128D240A167E
:102230000D300C1E192999000A300C1E1D29990019
:102240003C2F0A12AC2D0A163030831603172202D7
:10225000003A031D3129831203138813342983168E
:1022600003178312031388173030831603172402D1
:10227000003A031D4129831203138812442983164F
:1022800003178312031388163030831603172602B0
:10229000003A031D5129831203130813542983168E
:1022A000031783120313081730308316031728020D
:1022B000003A031961298312031305126429831656
:1022C00003178312031305166C300C1E6529990041
:1022D0000D300C1E692999000A300C1E6D299900D9
:1022E0003C2F831603172208303A83120313031975
:1022F0008029013A0319BA29033A0319F4291F2A3C
:102300006D300C1E812999002C300C1E85299900F6
:102310008316031754080313A0000330A1000A1208
:10232000831200260A162C300C1E9429990083165D
:10233000031752080313A0000330A1000A128312EE
:1023400000260A162C300C1EA329990083160317A9
:1023500053080313A0000330A1000A1283120026C1
:102360000A160D300C1EB22999000A300C1EB6292F
:1023700099001F2A6D300C1EBB2999002C300C1EB1
:10238000BF2999008316031757080313A0000330D1
:10239000A1000A12831200260A162C300C1ECE2928
:1023A00099008316031756080313A0000330A100F9
:1023B0000A12831200260A162C300C1EDD29990001
:1023C0008316031755080313A0000330A1000A1257
:1023D000831200260A160D300C1EEC2999000A30D3
:1023E0000C1EF02999001F2A6D300C1EF52999004A
:1023F0002C300C1EF9299900831603175908031372
:10240000A0000330A1000A12831200260A162C3005
:102410000C1E082A99008316031758080313A000FE
:102420000330A1000A12831200260A160D300C1E7A
:10243000172A99000A300C1E1B2A99001F2A3C2FCC
:102440006E300C1E212A99002C300C1E252A990072
:10245000831603175C080313A0000330A1000A12BF
:10246000831200260A162C300C1E342A990083167B
:1024700003175A080313A0000330A1000A128312A5
:1024800000260A162C300C1E432A990083160317C7
:102490005B080313A0000330A1000A128312002678
:1024A0000A162C300C1E522A9900831603175F0857
:1024B0000313A0000330A1000A12831200260A169B
:1024C0002C300C1E612A9900831603175E08031333
:1024D000A0000330A1000A12831200260A162C3035
:1024E0000C1E702A9900831603175D080313A000C1
:1024F0000330A1000A12831200260A162C300C1E8B
:102500007F2A99008316031761080313A000033084
:10251000A1000A12831200260A162C300C1E8E2AE5
:1025200099008316031760080313A0000330A1006D
:102530000A12831200260A160D300C1E9D2A9900DD
:102540000A300C1EA12A99003C2F6F300C1EA62ABF
:1025500099002C300C1EAA2A9900831603175408E0
:102560000313A0000330A1000A12831200260A16EA
:102570002C300C1EB92A9900831603175208031336
:10258000A0000330A1000A12831200260A162C3084
:102590000C1EC82A99008316031753080313A000C2
:1025A0000330A1000A12831200260A162C300C1EDA
:1025B000D72A99008316031757080313A000033086
:1025C000A1000A12831200260A162C300C1EE62ADD
:1025D00099008316031756080313A0000330A100C7
:1025E0000A12831200260A162C300C1EF52A9900B6
:1025F0008316031755080313A0000330A1000A1225
:10260000831200260A162C300C1E042B9900831608
:10261000031759080313A0000330A1000A12831204
:1026200000260A162C300C1E132B99008316031754
:1026300058080313A0000330A1000A1283120026D9
:102640000A160D300C1E222B99000A300C1E262B68
:1026500099003C2F831603172208303A8312031384
:102660000319392B013A0319732B033A0319AD2BC4
:10267000D82B70300C1E3A2B99002C300C1E3E2BA0
:102680009900831603175C080313A0000330A10010
:102690000A12831200260A162C300C1E4D2B9900AC
:1026A000831603175A080313A0000330A1000A126F
:1026B000831200260A162C300C1E5C2B9900831600
:1026C00003175B080313A0000330A1000A12831252
:1026D00000260A160D300C1E6B2B99000A300C1EBA
:1026E0006F2B9900D82B70300C1E742B99002C3056
:1026F0000C1E782B9900831603175F080313A000A4
:102700000330A1000A12831200260A162C300C1E78
:10271000872B9900831603175E080313A00003306C
:10272000A1000A12831200260A162C300C1E962BCA
:102730009900831603175D080313A0000330A1005E
:102740000A12831200260A160D300C1EA52B9900C2
:102750000A300C1EA92B9900D82B70300C1EAE2B02
:1027600099002C300C1EB22B9900831603176108B8
:102770000313A0000330A1000A12831200260A16D8
:102780002C300C1EC12B990083160317600803130D
:10279000A0000330A1000A12831200260A160D3091
:1027A0000C1ED02B99000A300C1ED42B9900D82B6C
:1027B0003C2F0A12482E0A16831603172208031309
:1027C000A5000A128312AE260A167808F300730ECB
:1027D0008316A000F030A005031723080313A500FB
:1027E0000A128312AE260A16780883162007F30011
:1027F00011141118F92B7308A3000A1283125E2515
:102800000A168316031725080313A5000A1283125C
:10281000AE260A167808F400740E8316A000F03075
:10282000A005031726080313A5000A128312AE267B
:102830000A16780883162007F4007408A3000A1209
:1028400083125E250A168316031728080313A500B2
:102850000A128312AE260A167808F400740E831644
:10286000A000F030A005031729080313A5000A12E1
:102870008312AE260A16780883162007F4009114F6
:102880009118402C01307307A000A3000A12831294
:102890005E250A1672300C1E4B2C99007408013C00
:1028A0000318682C0130F7000A1270250A16780800
:1028B000F5002C300C1E5A2C990075088316A000C8
:1028C0000330A1000A12831200260A16F4034E2CCC
:1028D000F7010A1270250A167808F5002C300C1E34
:1028E0006F2C990075088316A0000330A1000A120E
:1028F000831200260A168316111511197D2C0D302E
:1029000083120C1A852C8316802C99000A300C1E19
:10291000872C99003C2F0A12BF2E0A160A12172F75
:102920000A160A12312F0A168316031722080313F8
:10293000A5000A128312AE260A167808F400740E57
:102940008316A000F030A005031723080313A50089
:102950000A128312AE260A16780883162007F4009E
:1029600011141118B12C7408A3000A1283125E25E9
:102970000A168316031725080313A5000A128312EB
:10298000AE260A167808F400740E8316A000F03004
:10299000A005031726080313A5000A128312AE260A
:1029A0000A16780883162007F4007408A3000A1298
:1029B00083125E250A168316031728080313A50041
:1029C0000A128312AE260A167808F400740E8316D3
:1029D000A000F030A005031729080313A5000A1270
:1029E0008312AE260A16780883162007F4007408AE
:1029F000A3000A1283125E250A16831611151119F7
:102A0000FF2C773083120C1A072D8316022D9900A4
:102A10000D300C1E092D99000A300C1E0D2D990049
:102A20003C2F0A12B12F0A1683160317220803132C
:102A3000A5000A128312AE260A167808F400740E56
:102A40008316A000F030A005031723080313A50088
:102A50000A128312AE260A16780883162007F4009D
:102A600011141118312D7408A3000A1283125E2567
:102A70000A168316031725080313A5000A128312EA
:102A8000AE260A167808F400740E8316A000F03003
:102A9000A005031726080313A5000A128312AE2609
:102AA0000A16780883162007F4007408A3000A1297
:102AB00083125E250A168316031728080313A50040
:102AC0000A128312AE260A167808F500750E8316D0
:102AD000A000F030A005031729080313A5000A126F
:102AE0008312AE260A16780883162007F5007508AB
:102AF000A3000A1283125E250A16F60175087602F3
:102B00000318B22D0B30760776077607A03E8400B7
:102B1000831700088316A300A5000A128312AE26AD
:102B20000A167808F400740E8316A000F030A00591
:102B30000C30760776077607A03E840083170008DE
:102B4000A400A5000A128312AE260A16780883167E
:102B50002007F4007408A3000A1283125E250A16E7
:102B6000F60A7E2D831611151119B42D79308312B2
:102B70000C1ABC2D8316B72D99000D300C1EBE2DDE
:102B800099000A300C1EC22D99003C2F0A12C02F4A
:102B90000A16031083160317630D62040313A000C3
:102BA0000317640DF700F70DFC30F70577080313E2
:102BB0002004A1000317650DF700F70DF70DF8309D
:102BC000F705770803132104A200263083120C1A9C
:102BD000EB2D8316E62D99002A080C1EED2D990089
:102BE0002B080C1EF12D9900831603175C08831225
:102BF00003130C1AFE2D83160317F72D9900831665
:102C000003175A08831203130C1A092E831603178D
:102C1000022E9900831603175B08831203130C1A04
:102C2000142E831603170D2E9900831603175F08C1
:102C3000831203130C1A1F2E83160317182E9900E4
:102C4000831603175E08831203130C1A2A2E8316A9
:102C50000317232E9900831603175D0883120313AD
:102C60000C1A352E831603172E2E99008316031780
:102C70006108831203130C1A402E83160317392E92
:102C80009900831603176008831203130C1A4B2E46
:102C900083160317442E99008316031754088312D2
:102CA00003130C1A562E831603174F2E9900831602
:102CB00003175208831203130C1A612E831603178D
:102CC0005A2E9900831603175308831203130C1A04
:102CD0006C2E83160317652E990083160317570869
:102CE000831203130C1A772E83160317702E990084
:102CF000831603175608831203130C1A822E8316A9
:102D000003177B2E990083160317550883120313AC
:102D10000C1A8D2E83160317862E9900831603171F
:102D20005908831203130C1A982E83160317912E39
:102D30009900831603175808831203130C1AA32E45
:102D4000831603179C2E99008316220883120C1AEF
:102D5000AB2E8316A62E990031080C1EAD2E9900BD
:102D600001300C1EB12E990033300C1EB52E990087
:102D70000D300C1EB92E99000A300C1EBD2E990084
:102D80003C2F83160317210883120313AA0083160E
:102D90000317220883120313AB00831603172318AB
:102DA000D72E831203138813DA2E83160317831288
:102DB0000313881783160317A318E42E8312031333
:102DC0008812E72E831603178312031388168316BF
:102DD00003172319F12E831203130813F42E8316FD
:102DE000031783120313081783160317A31DFE2E60
:102DF000831203130512012F831603178312031383
:102E000005162A300C1E022F99000D300C1E062FBD
:102E100099000A300C1E0A2F99003C2F00302D1A01
:102E200001308316A000213083120C1A192F83164B
:102E3000142F99008316200883120C1A212F831651
:102E40001C2F99000D300C1E232F99000A300C1EE8
:102E5000272F99002D1E2D2F2D123C2F0A128A1577
:102E600000280A168A110A128A156F280A168A1172
:102E70000A12D1270A163C2FAE018C128A110A12AF
:022E80002D28FB
:0E360200840183131F30830583161F149F1449
:103610001F159F110A3099002630980090308312B0
:103620009800A915290883168700831229162908EE
:10363000831687003130930028308312940083165C
:1036400094171413FF308312A900AA01AB01AC0137
:103650002D14AD142D15AD152D12AD12AE012D1377
:10366000AD132F10AF102F11AF112F12AF122F1358
:10367000AF133010B0103011B011B101B201B3016D
:10368000B401B501B601B701B801B901BA018F01A2
:103690008E010A12D0280A16003087180130003A2D
:1036A000031D7C2B003007190130003A031D7C2BD1
:1036B0000030871A0130003A031D7C2B00300718B8
:1036C0000130003A031D682BFF30C200C1007B2B84
:1036D000FF3003178D001A308F0083168C170C14DF
:1036E0000000000083120E08FA000C080313C1004A
:1036F00018307A07C2007F2B0A12962B0A168316FF
:103700008C128312410F872B420F872B5A2EB01A2F
:10371000A22B0F08FA000E08F7000F087A02031D0B
:10372000892B7708C8007A08C90049087C3C03182F
:10373000A22BFF3A031DA02B4808003C0318A22B24
:10374000B016B62BB01EB62B0F08FA000E08F70005
:103750000F087A02031DA42B7708C8007A08C90055
:1037600049087C3C031CB62BBE0AB012C7010A12E2
:10377000DF2D0A164208C0004108BF00C401C50180
:103780004610C61046124611C6113F0803178D0099
:103790000313400803178F0083168C170C140000C6
:1037A000000083120E08FA000C080313C7007A0801
:1037B000C8004708FC3E0318522C043E682EBF0A7E
:1037C0000319C00A3F0803178D00031340080317AD
:1037D0008F0083168C170C140000000083120E0853
:1037E000FA000C080313C7007A08C8004708C40091
:1037F000522CBF0A0319C00A3F0803178D00031398
:10380000400803178F0083168C170C14000000006B
:1038100083120E08FA000C080313C7007A08C800C8
:103820004708C500522CBF0A0319C00A3F080317F6
:103830008D000313400803178F0083168C170C1498
:103840000000000083120E08FA000C080313C700E2
:103850007A08C8004708C30043184614C318C614A2
:1038600043194615C319C615522CBF0A0319C00ABD
:103870003F0803178D000313400803178F008316BA
:103880008C170C140000000083120E08FA000C08BC
:103890000313C7007A08C8004708C300430B512C24
:1038A0004616522CBF0A0319C00A3F0803178D00A1
:1038B0000313400803178F0083168C170C140000A5
:1038C000000083120E08FA000C080313C7007A08E0
:1038D000C8004708FF3C031DC52B4408D700450816
:1038E000D8000A1291230A160030461A0130C70088
:1038F000D7000A1257230A16003046180130C700B5
:10390000D7000A1283230A160030C6180130C700F8
:10391000D7000A128A230A164619902C0613912CF6
:103920000617C619952C8613962C8617BF0A0319FD
:10393000C00A3F0803178D000313400803178F00C8
:1039400083168C170C140000000083120E08FA0076
:103950000C080313C7007A08C8004708FF3C031986
:103960005A2E30163F0803178D0003134008031723
:103970008F0083168C170C140000000083120E08B1
:10398000FA000C080313C7007A08C8004708BB00F8
:103990003B0FCB2C182E3B08043A0319362D013A65
:1039A0000319362D033A0319362D013A0319362D22
:1039B0000F3A0319362D013A0319362D033A03192C
:1039C000362D013A0319362D073A03195C2D013AB9
:1039D00003195C2D033A03195C2D013A03195C2D80
:1039E0001F3A03195C2D013A03195C2D033A0319A0
:1039F0005C2D013A03195C2D073A0319822D013A17
:103A000003199E2D033A0319A22D923A0319C22DD0
:103A1000013A0319C22D033A0319C22D013A0319C1
:103A2000C22D0F3A0319C22D013A0319C22D033AD0
:103A30000319C22D013A0319C22D073A0319EB2DC0
:103A4000013A0319EB2D033A0319EB2D013A03193F
:103A5000EB2D1F3A0319EB2D013A0319EB2D033A15
:103A60000319EB2D013A0319EB2D142EBF0A03198C
:103A7000C00A04303B02BD003D08D7000A125023A3
:103A80000A167808C7003F0803178D000313400883
:103A900003178F0083168C170C140000000083128C
:103AA0000E08FA000C080313C8007A08C900480879
:103AB000470203183012142EBF0A0319C00A0C3033
:103AC0003B02BD003D08C7000A12E8250A16780827
:103AD000C7003F0803178D000313400803178F002A
:103AE00083168C170C140000000083120E08FA00D5
:103AF0000C080313C8007A08C900480847020318D5
:103B00003012142EBF0A0319C00A3F0803178D0094
:103B10000313400803178F0083168C170C14000042
:103B2000000083120E08FA000C080313C7007A087D
:103B3000C80047083E02031C3012142EBF0A0319A6
:103B4000C00A142EBF0A0319C00A0030061801303B
:103B5000C7003F0803178D000313400803178F00A9
:103B600083168C170C140000000083120E08FA0054
:103B70000C080313C8007A08C90048084702031D4F
:103B80003012142EBF0A0319C00A3B087F39BD004A
:103B90000430BD023D08D7000A1250230A167808E7
:103BA000C7003F0803178D000313400803178F0059
:103BB00083168C170C140000000083120E08FA0004
:103BC0000C080313C8007A08C90048084702031DFF
:103BD000031C3012142EBF0A0319C00A3B087F3998
:103BE000BD000C30BD023D08C7000A12E8250A16C8
:103BF0007808C7003F0803178D0003134008031718
:103C00008F0083168C170C140000000083120E081E
:103C1000FA000C080313C8007A08C90048084702D4
:103C2000031D031C3012142EBF0A0319C00AB22C44
:103C3000BF0A0319C00A301E552E3F0803178D0016
:103C40000313400803178F0083168C170C14000011
:103C5000000083120E08FA000C080313C7007A084C
:103C6000C80001303F07C9004008CA000318CA0A4B
:103C7000490803178D0003134A0803178F008316A2
:103C80008C170C140000000083120E08FA000C08B8
:103C90000313CA007A08CB004A08C100183047074E
:103CA000C2008F018E01BE01B0120230BF0703189F
:103CB000C00A992C83168C1602308312C700F93083
:103CC000DA000A12DB210A16C70B5F2E7F2B630076
:103CD0000A108A140A158207DF2BF92B132C352CB6
:02400E003A3D39
:00000001FF
